:100000000C946F020C94A7020C94A7020C94A70204
:100010000C94A7020C94A7020C94A7020C94A702BC
:100020000C94A7020C94A7020C94E2220C94B42323
:100030000C94691D0C94A7020C94A7020C94A702BF
:100040000C94A7020C94A7020C94A7020C94A7028C
:100050000C94A7020C94F21D0C94A7020C94A70216
:100060000C94A7020C94A7020C94A7020C94A7026C
:100070000C94A7020C94A7020C94A7020C94A7025C
:100080000C94A7020C94A7020C94A7020C94A7024C
:100090000C94A7020C94A7020C94A7020C94A7023C
:1000A0000C94A7020C94A7020C94A702DD05DD05B1
:1000B0000906090677069506760776079A06020767
:1000C00013071307AF15B215DC15EF15F715021658
:1000D0000516051605164D164D160A160D1612169E
:1000E0001F162C162F1633164016AE162017B616EE
:1000F00080168416BA168716BD16C81692161617DD
:100100009616CC169A16D016FA169E16D416041702
:10011000A416DA16E4168B16C1168E16C416A91686
:10012000DF16F016101712177C16B2162917A11831
:100130009718A418F418F818F818F418F818F818FC
:10014000C518F818CF18D918F818F818F818F818AA
:10015000F418F818F818F418F818B218F818F8186D
:10016000E918E918E918E918E918E918E918E91887
:10017000E918F618F818A1189418F818F818F818CB
:10018000F818F818F818F818F818F818F818F618F1
:10019000F818F818F418F818E718E718E718E71827
:1001A000E718E718E718E718E718F6189C1BA21BD2
:1001B000901B961BA81BAE1BB41B1C2443243B2581
:1001C00043243B258F24B2243B25092518255300C1
:1001D0005400550056005F006000610057005C004D
:1001E0005D005E00570059005A005B005800620035
:1001F00062006300580001000100010001000100DD
:1002000001000100010001000100010001000100E6
:1002100001000100010001000100010001000100D6
:1002200001000100010001000100010001000100C6
:1002300001000100010001000100010001000100B6
:1002400001000100010001000100010001000100A6
:100250000100010001000100010001000100010096
:100260000100010001000100010001000100000087
:100270000000000000002A2B280000000000000001
:1002800000000000000000000029000000002C1EFB
:100290003420212224342627252E362D3738271EB8
:1002A0001F202122232425263333362E37381F04DE
:1002B00005060708090A0B0C0D0E0F101112131476
:1002C00015161718191A1B1C1D2F3130232D350434
:1002D00005060708090A0B0C0D0E0F101112131456
:1002E00015161718191A1B1C1D2F3130354C00001C
:1002F00000000000000000000000000000000000FE
:1003000000000000000000000000000000000000ED
:1003100000007E0F00D4FFFFFFC7000000780C0331
:1003200053006F00790075007A0000002603610019
:10033000690030003300200044006500730069004C
:1003400067006E00200053007400750064006900AF
:100350006F0000000403090409025B00030100A010
:10036000FA09040000010301010009211101000143
:10037000224000070581030800010904010002036F
:10038000000000092111010001222200070582035B
:1003900020000107050303200001090402000103F6
:1003A00000000009211101000122B60007058403A5
:1003B000200001120100020000000803A118000142
:1003C00000010200010660FF0961A1010962150038
:1003D00026FF009520750881020963150026FF009D
:1003E000952075089102C005010902A10185020945
:1003F00001A10005091901290815002501950875B5
:100400000181020501093009311581257F950275A9
:1004100008810609381581257F9501750881060533
:100420000C0A38021581257F950175088106C0C028
:1004300005010980A101850319012AB700150126CC
:10044000B700950175108100C0050C0901A1018557
:100450000419012AA002150126A002950175108138
:1004600000C005010906A1018506050719E029E775
:10047000150025019508750181020507190029EF6E
:100480001500250195F0750181020508190129055E
:10049000950575019102950175039101C00501094A
:1004A00006A101050719E029E71500250195087542
:1004B0000181029501750881010507190029FF15C1
:1004C0000026FF0095067508810005081901290519
:1004D000950575019102950175039101C0001124E4
:1004E0001FBECFEFDAE0DEBFCDBF04B603FE18C0FB
:1004F0008091940290919502A0919602B0919702FA
:100500008730904BA740B04B59F410929402109250
:1005100095021092960210929702E0E0F8E3099596
:1005200011E0A0E0B1E0EEE5FCE402C005900D9220
:10053000A639B107D9F722E0A6E9B1E001C01D92C2
:10054000A439B207E1F70E9451120C942D260C94A5
:10055000000084E008958430C0F46530B0F4443085
:10056000A0F4E62FF0E095E0899FE00DF11D112445
:10057000EE0FFF1FEE0FFF1FE40FF11DEE0FFF1F29
:10058000E253FE4F85919491089580E090E00895A4
:1005900081E0089581E008950E94CA0208950895B7
:1005A0000E94CF020895A5E0B0E0E9EDF2E00C94DE
:1005B000992549835A8330919D0189819A8131110E
:1005C00014C0662359F0222349F00E943009182FE5
:1005D000682F89819A810E940C0903C00E941E091C
:1005E000182F69817A81812F04C00E9430096981A6
:1005F0007A810E94DF0F2596E3E00C94B525FC017B
:10060000262F408151816281738184810E94D302AF
:10061000089581E00895CF93DF93EC0160E00E949C
:10062000FF02BE010E94D002DF91CF910895E1E068
:10063000F0E0DF0102C0AA0FBB1F6A95E2F7BD011F
:10064000DF0102C0AA0FBB1F4A95E2F7AD01462B9E
:1006500001C0EE0F2A95EAF7942F9823491302C0A0
:100660008E2B0895E0958E230895242F462F682F12
:100670008091A7010E9417030E946D0808950E94AF
:10068000201108950E941A11089508950E94F907F3
:100690000E9445032FEF84E39CE02150804090406E
:1006A000E1F700C0000008950E9446030E94181E52
:1006B00008950E9446030E943C1E08950F931F93C5
:1006C000CF93DF938C0161E00E94FF02EC01B8013F
:1006D0000E945515882309F449C0B801CE010E9433
:1006E000CC02882309F442C0B801CE010E94841BC9
:1006F0008823E1F1B801CE010E9458168823B1F198
:10070000B801CE010E94EA1A882381F1F8018281A2
:10071000882341F1C3308CE7D807D1F040F4C115EC
:10072000FCE7DF0791F0C130DC47A1F01BC0CB35FF
:10073000ECE7DE07A9F0CC35FCE7DF0771F0CA353E
:10074000DC4781F40E94660D0DC00E9454030EC068
:100750000E946E0D0E94590309C00E945C0D02C0E8
:100760000E946A0DC8010E94C80201C080E0DF91AA
:10077000CF911F910F9108950E94421D0E94E603A0
:1007800008950E94EA030E944B1D089508950E9457
:10079000C603089581E008950895CF93DF93D82F7D
:1007A0000E94CA03C82F882319F08D2F0E94CC0302
:1007B0008C2FDF91CF9108950895CF93C82F0E9479
:1007C000C7038C2F0E94CD03CF91089580E00E9433
:1007D000DD0308950E94D11B0E94DD030895CF938D
:1007E0000E94D11BC82F80919801C81779F0C0933F
:1007F00098010E94D71D6093990170939A0180938C
:100800009B0190939C018C2F0E94DD03CF91089552
:10081000ABE0B0E0EEE0F4E00C949A254F8358870B
:1008200069877A878B8761110E94A40C9E012F5FD4
:100830003F4F86E0F90111928A95E9F785E0FE01C4
:100840003796D90101900D928A95E1F789819A81B5
:100850004C815D81452B31F09F3F31F491E08F3F1A
:1008600019F403C091E001C090E090FF09C04981F4
:100870005A816B817C818D819E810E94D00B05C045
:10088000C9010E9409038111F2CF2B96E2E00C947A
:10089000B625FC01808191810E945D09089566233F
:1008A00019F00E94D61202C00E9431130E94A813B0
:1008B0000895CF93882309F4A9C0C82F8238C1F4C2
:1008C0000E94D11B81FDA2C069E38091000190913B
:1008D00001010E94E61C0E94C80C2FEF87EE93E0F6
:1008E000215080409040E1F700C0000069E319C04A
:1008F000833801F50E94D11B80FD88C063E580919B
:100900000001909101010E94E61C0E94C80C2FEF8B
:1009100081EE94E0215080409040E1F700C000005B
:1009200063E580910001909101010E94F41C0E94F6
:10093000C80C6CC08438C1F40E94D11B82FD66C013
:1009400067E480910001909101010E94E61C0E94E1
:10095000C80C2FEF81EE94E0215080409040E1F7E9
:1009600000C0000067E4DDCF8CEF8C0F813AF8F413
:100970008C2F0E94FF18811149C06C2F80910001BB
:10098000909101010E94661C882349F06C2F809190
:100990000001909101010E94F41C0E94C80C6C2F70
:1009A00080910001909101010E94E61CC0CF80E27D
:1009B0008C0F883048F4C77081E001C0880FCA9559
:1009C000EAF70E94870CB3CFEBE5EC0FE33040F47D
:1009D000F0E0EB5BFE4F808190E00E94061C16C0A9
:1009E000E8E5EC0FE93150F4F0E0EE0FFF1FED5EAB
:1009F000FE4F808191810E942B1C08C083E38C0FE5
:100A0000833120F461E08C2F0E944F04CF91089530
:100A1000882309F468C0823879F40E94D11B81FFD1
:100A200062C069E380910001909101010E94E61C7F
:100A30000E94C80C69E310C08338B9F40E94D11B2E
:100A400080FF51C063E580910001909101010E94F7
:100A5000E61C0E94C80C63E58091000190910101A1
:100A60000E94F41C0E94C80C0895843879F40E94F6
:100A7000D11B82FF38C067E4809100019091010191
:100A80000E94E61C0E94C80C67E4E6CF9CEF980F1A
:100A9000913A10F4682FE0CF90E2980F983050F41C
:100AA000877091E001C0990F8A95EAF7892F0E941B
:100AB0008D0CD8CF9BE5980F933028F480E090E020
:100AC0000E94061C089598E5980F993128F480E05B
:100AD00090E00E942B1C089593E3980F933118F433
:100AE00060E00E944F0408951F93CF93DF93182F67
:100AF000EB010E945904209741F08FE99FE0019794
:100B0000F1F700C000002197F6CF812F0E94080561
:100B1000DF91CF911F910895893319F060E070E063
:100B200002C060E570E00E9474050895882321F0FA
:100B30000E94870C0E94C80C0895882321F00E940F
:100B40008D0C0E94C80C0895A0E0B0E0EAEAF5E040
:100B50000C9494257C01162FC72FFC01D2810581AE
:100B600002950F700E947D0C8823B9F0DD23A9F057
:100B70008C2F807F803421F080E2810F883068F0F4
:100B80008091780282FF09C082E00E942A0D0E94B3
:100B90007D0C91E0D82ED92601C0D12CCC2EC29448
:100BA0008FE0C8228C2D90E08C30910508F09EC11A
:100BB000FC01EA5AFF4F0C947D258C2F807FCF706B
:100BC000882311F0C295C07FDD2399F0CC2309F46E
:100BD00079C180E2810F883010F0111104C08C2F90
:100BE0000E94870C03C08C2F0E94970C0E94C80C97
:100BF00069C1812F0E940805CC2309F477C180E2E6
:100C0000810F883038F1112329F18C2F0E949D0C1F
:100C100024C08C2F807FCF70803211F0C295C07FAE
:100C2000112319F01130D1F143C08091780282FD77
:100C300017C0DD2349F0CC2329F08C2F0E94870CAC
:100C40000E94C80C80E03FC180E00E940805CC23D0
:100C500009F44CC18C2F0E948D0C0E94C80C46C117
:100C6000DD2371F0002341F0013031F40E94A70C24
:100C70008C2B0E94B10C3AC10E94A70C8C2B23C074
:100C8000011103C00E94BE0C2EC0013009F42EC118
:100C90008C2F0E949D050E94BE0C28C1DD2321F0EF
:100CA000063008F023C10EC0053008F01FC11BC07C
:100CB000DD2361F0002331F0F701858180FF02C15F
:100CC0008F7085838C2F0E94960510C1002359F0E8
:100CD000193309F008C1FFEF27EE83E0F1502040FF
:100CE0008040E1F7FEC08C2F0E949D05FFC08C2F35
:100CF00086958695837019F0813061F0F7C0DD2309
:100D000021F0812F9C2F937002C080E090E00E9420
:100D1000061CF4C0DD2321F0812F9C2F937002C0AC
:100D200080E090E00E942B1CE9C06D2F812F0E9473
:100D30004F04E4C08C2F837079F5D111DBC0412FB3
:100D4000429546954770440F440F212F2F70042E73
:100D500001C0220F0A94EAF714FF08C08FE090E068
:100D600001C0880F4A95EAF7809501C080E0C695DA
:100D7000C695C370822BC23049F058F4C13019F0C7
:100D80000E945E08B7C00E945808B4C00E94640860
:100D9000B1C00E945508AEC0DD2319F08C2F8170C0
:100DA00001C08695882309F4A5C0412F4295469538
:100DB0004770440F440F212F2F70042E01C0220FC3
:100DC0000A94EAF714FF08C08FE090E001C0880F92
:100DD0004A95EAF7809501C080E0C695C695C37034
:100DE000822BC23049F058F4C13019F00E94AA0891
:100DF00081C00E94A4087EC00E94B0087BC00E94EF
:100E00006D0878C0CF70DD2339F08C2F0E947F08E9
:100E1000812F0E9496056EC0812F0E949D058C2F08
:100E20000E948B0867C0123F21F128F4103F41F067
:100E3000113FC1F043C0133F19F1143F79F03EC098
:100E4000DD2341F0053008F051C08C2F8F710E94D6
:100E500098084CC0063008F049C0F7CF809178025E
:100E600082FD18C0DD2339F08C2F8F710E947F081E
:100E70003DC0DD23C9F38C2F8F710E948B0836C0D3
:100E8000DD2329F08C2F8F710E9476082FC00E94DD
:100E900072082CC0DD2349F0CF718C2F0E947F088F
:100EA00063E08C2F0E940C0D21C081E00E942A0D6E
:100EB0000230E0F082E00E942A0D18C0DD2331F0FC
:100EC000002391F2812F0E94590410C0002399F24F
:100ED000193349F49FEFE7EEF3E09150E040F04022
:100EE000E1F700C00000812F0E94080588EF8C0DFB
:100EF000843020F40E94D11B0E94DD03DD2089F0A4
:100F00000E94790C80FD0DC0F70112820E94730CC3
:100F10000E947F08C7010E94AE070E94730C0E94C6
:100F20008B08CDB7DEB7E8E00C94B0250F931F9384
:100F3000CF93DF93EC01688179818A810E946809EF
:100F40008C010E94B6080E944808B801CE010E9498
:100F5000A405DF91CF911F910F910895CF93DF9357
:100F6000EC01988189812B813C81232B31F08F3FCB
:100F700031F481E09F3F19F403C081E001C080E0BB
:100F800080FD1AC0CE010E945E0381110FC00E9435
:100F90007D0C882389F08A81882371F08091780202
:100FA00082FF0AC082E00E942A0D06C0CE010E9484
:100FB0009607CE010E940B03DF91CF91089580E048
:100FC00090E00E94061C80E090E00E942B1C0E9492
:100FD000A40C0E94C80C0E94C7130E94A813089575
:100FE00080910001909101010E94021D0E94DF0783
:100FF00008950E94940C0E94F007089592959F70A6
:10100000963079F010F4925001C09A50923068F402
:10101000803F69F018F4883E40F409C0843F29F409
:1010200006C0883E20F0813F11F080E0089581E005
:101030000895FC019081818123813481232B31F03B
:101040008F3F31F481E09F3F19F403C081E001C07C
:1010500080E080FD07C0808191810E945D090E942F
:10106000FE07089580E00895A5E0B0E0EAE3F8E027
:101070000C949A252596E2E00C94B625A6E0B0E003
:10108000E4E4F8E00C949A252696E2E00C94B62568
:10109000089508950E94490808950E944A080895F5
:1010A0000E944D088093A80108950E945008089559
:1010B0009091A801892B0E94500808959091A80151
:1010C00089230E94500808959091A80189270E94C1
:1010D000500808950E94490808950E946A08809364
:1010E000A701089580E00E946D08089591E001C075
:1010F000990F8A95EAF7892F0E946D08089521E0DB
:1011000030E001C0220F8A95EAF78091A701822B77
:101110000E946D08089521E030E001C0220F8A95F9
:10112000EAF720958091A70182230E946D08089517
:1011300021E030E001C0220F8A95EAF78091A701F3
:1011400082270E946D0808959091A701892B0E9423
:101150006D0808959091A70189230E946D08089554
:101160009091A70189270E946D0808950895962FF0
:101170009770A1E001C0AA0F9A95EAF793E07695DF
:1011800067959A95E1F7FB01EE0FFF1F6E0F7F1F2A
:10119000FA01E60FF71F40E050E0682F70E0908101
:1011A0009B01042E02C0369527950A94E2F7217020
:1011B000219529272A23292721934F5F5F4F433009
:1011C000510569F708959B01782F777043E0969554
:1011D00087954A95E1F7FC01EE0FFF1F8E0F9F1FC9
:1011E000F901E80FF91F40E050E080E0219130E084
:1011F000072E02C0369527950A94E2F7217033270F
:10120000042E01C0220F0A94EAF7822B4F5F5F4F32
:101210004330510559F70895282F953070F48430E4
:1012200060F4862F622F70E024E0929F600D711DA4
:1012300011244EE951E00E94B7080895953070F4EA
:10124000843060F4292F90E06EE971E034E0239F50
:10125000800D911D11240E94E308089580E00895F7
:10126000CF92DF92FF920F931F93CF93DF936C0186
:101270000091A7018091A801082BC7E0D0E010E001
:10128000C8010C2E02C0959587950A94E2F780FD5F
:1012900004C02197A8F7F12C07C0FC2EB6018C2FB3
:1012A0000E94EB0F0197A9F38F2DDF91CF911F9132
:1012B0000F91FF90DF90CF900895CF93DF93EC01D3
:1012C0000E943009BE010E94EB0FDF91CF9108957B
:1012D0001F93CF93DF93EB0190919D01992321F010
:1012E000CB010E945D0913C0882349F0CB010E9405
:1012F0003009182F682FCE010E940C0904C0CB01C1
:101300000E941E09182FBE01812F0E94EB0FDF9152
:10131000CF911F9108951F93CF93DF93C091A9019F
:1013200016E08091AA01C81799F0D0E01C9FF00147
:101330001D9FF00D1124E555FE4F408151816281C2
:101340007381848195810E943E082196C770E9CF00
:10135000DF91CF911F9108954091DB015091DC0105
:101360006091DD017091DE018091DF019091E001DB
:101370000E943E0808950F931F93CF93DF938091AF
:10138000E00182958F7009F05AC08091DD018823B9
:1013900009F455C08091A9011091AA016091DB0167
:1013A0007091DC01C091DE01D091DF0191E06F3FCF
:1013B00009F090E0292F06E0811709F440C020973A
:1013C00021F07F3F21F030E003C031E001C0322F37
:1013D00090E030FD31C0089FF001099FF00D11240D
:1013E000DF01A555BE4F11963C911197371324C0CC
:1013F0003C91361321C012963C91129731111CC0BA
:1014000013964D915C9114974C1B5D0B483C510514
:1014100098F48091E0018F7080618093E001E05545
:10142000FE4F80818F70806180838BED91E00E9400
:10143000AE070E948B0903C001968770BDCFDF9174
:10144000CF911F910F910895A1E1B0E0EAE2FAE097
:101450000C9491258C0185E0F801DE011D96019028
:101460000D928A95E1F7F801E2809091DB0160919D
:10147000DC012091DE013091DF012115310531F0D1
:101480006F3F31F481E09F3F19F403C081E001C058
:1014900080E0F82FF1709F2E80FD40C1F80140815F
:1014A0005181A380B4808BEDC82E81E0D82EF090BE
:1014B000DD01F501E21BF30BFF2009F4DAC0809196
:1014C000E001E83CF10508F096C0282F207F09F0E4
:1014D00053C0561313C0491311C0FE2CE1100EC0A7
:1014E0008F7080618093E0010E94AC09C6010E9468
:1014F000AE078091E001F80185834DC1A114B104CC
:1015000031F05F3F31F481E04F3F19F403C081E0D7
:1015100001C080E080FD03C081E08E2502C080E034
:1015200090E0F82FF170FF2E80FF1CC08091A90180
:101530002091AA0136E0821709F40BC190E0389F90
:10154000F001399FF00D1124E555FE4F61815613CE
:1015500006C06081461303C06281E61203C0019693
:101560008770E9CFFE2CEE2009F415C18091E001CF
:1015700081608093E00154C0561306C0491304C033
:10158000E11002C0F80199C0C8010E94190888231F
:1015900061F1EE2051F12091E001822F82958F7050
:1015A00090E0029774F08091DB019091DC019887C4
:1015B0008F831986BB86AA862C87CE0107960E9448
:1015C000AE0786E0F801ABEDB1E001900D928A958F
:1015D000E1F70E94BB090E94AC090AC0561711F13D
:1015E000C8010E94190881112CC0C8010E94AE07D1
:1015F000FF24F394D0C0282F207F81F77A2DB98A59
:10160000A88A6E2D89890E9434088BED91E00E9492
:10161000AE0786E0F60111928A95E9F70E94AC09BF
:10162000F12CB9C04913DCCFE110DACFF801858382
:10163000C8010E94AE0786E0F60111928A95E9F78B
:10164000AAC0EE2091F22091E001822F82958F7046
:1016500090E002970CF4B5CF8091DB019091DC0112
:101660009A8389831B82BD82AC822E83CE01019630
:10167000A6CFE83CF10508F044C0FE2CEE2009F4AA
:10168000B4CF561330C049132EC02091E00120FD85
:1016900021C0822F82958F70482F50E0411551054F
:1016A000C9F0F80125834F30510541F08F5F982F25
:1016B0009295907F822F8F70892B8583C8010E941D
:1016C000AE0786E0F801ABEDB1E001900D928A958E
:1016D000E1F73CC086E0F801ABEDB1E001900D927E
:1016E0008A95E1F758C0C8010E941908811169CF95
:1016F0008091E00181608093E001C8010E94AE0703
:101700004AC07A2DB98AA88A6E2D89890E94340828
:1017100086E0F60111928A95E9F718C0EE2009F4E7
:1017200064CFC8010E941908F82E882309F45DCF00
:1017300086E0F801ABEDB1E001900D928A95E1F7FA
:101740008BED91E00E9449040E94BB090E94AC0904
:1017500022C04D875E878D859E850E945D09292F59
:1017600022952F70223028F49F7039F0811105C026
:101770000BC0243028F49F7049F4805E883020F03C
:10178000C8010E94AE079F2CF92C05C0F801958175
:10179000907F99F7F9CF8F2D6196EBE00C94AD25F2
:1017A000ACE0B0E0E6EDFBE00C9499254F83588760
:1017B00069877A878B879C87CE0107960E94240AC7
:1017C0008823D1F09F8188852A853B85232B31F0A2
:1017D0008F3F31F481E09F3F19F403C081E001C0E5
:1017E00080E080FD47C04F81588569857A858B856B
:1017F0009C850E943E083EC086E0FE013796DE01D1
:10180000119601900D928A95E1F7FF81E8856A852E
:101810007B856115710531F0EF3F31F481E0FF3FC9
:1018200019F403C081E001C080E080FD23C0209155
:10183000AA0130E0C9010196877099274091A9015A
:1018400050E084179507F1F1F983EA837D836C8377
:1018500096E0929FD001939FB00D1124A555BE4FE5
:10186000FE01319601900D929A95E1F78093AA01BD
:101870000E948B0916E08091A9019091AA01891715
:1018800071F1189FC001112485559E4F0E94240AB2
:10189000882329F1E091A9011E9FF0011124E5554B
:1018A000FE4F4081518162817381848195810E94C4
:1018B0003E088091A90190E0019687709927809356
:1018C000A901D9CF0E94F9071092AA011092A9018B
:1018D000EBEDF1E086E0DF011D928A95E9F72C96A9
:1018E000E3E00C94B5258091010285958595859559
:1018F0000895809101028770089590910102977078
:1019000081E009F480E00895809124020895909187
:101910002402892B809324020895809590912402BB
:1019200089238093240208951092240208959091AF
:101930002302892B8093230208958095909123029E
:1019400089238093230208951092230208958091A1
:101950000202089508950E94AA0C08950E94AB0CFB
:1019600008959091780292FF08C090910202981712
:1019700021F0809302020E94AE0C08958091020231
:10198000882329F01092020280E00E94AE0C089594
:10199000CF93DF93E0910001F09101018091240247
:1019A0008083E0910001F0910101908180912302F8
:1019B000892B808380910202882381F0E0910001CD
:1019C000F09101019081892B808380910001909199
:1019D00001010E94501C81110E94BE0CC0910001A7
:1019E000D091010140E250E061EE71E0CE010E9431
:1019F000D525892B59F080E2FE01A1EEB1E00190DE
:101A00000D928A95E1F7CE010E94DE1BDF91CF9106
:101A100008950E94AA0C08959091780292FF11C037
:101A200098E0899F90011124262B209301020E94A7
:101A30007F08809101028595859585950E94090D05
:101A400008950E947F0808951092010280E00E948C
:101A5000090D08952091010280958223809301024F
:101A6000982F977099F430E0482F082E000C550BF2
:101A70002417350759F09091780292FF07C0859599
:101A8000859585950E948B080E94240D089590915C
:101A9000780292FB222720F9281769F080FB92F93F
:101AA0009093780280917702909178020E94900D35
:101AB00082E00E942A0D08958091780282FB882797
:101AC00080F991E089270E94470D089581E00E94E6
:101AD000470D089580E00E94470D08956FEF7FEF56
:101AE00080E090E00E941726089580E090E00E9438
:101AF000F325873E9E4F19F40E94E914089580E073
:101B0000089582E090E00E94EB25089583E090E044
:101B10000E94EB25089584E090E00E94F32508954B
:101B2000BC0184E090E00E9417260895AB01BC013F
:101B30008FE090E00E940B260895AB01BC0183E189
:101B400090E00E940B26089560E070E0CB010E94B7
:101B50009D0D089560E070E0CB010E94960D0E94FB
:101B6000A40D089567EE7EEF80E090E00E941726B6
:101B700060E082E090E00E94F92560E083E090E080
:101B80000E94F9251092A80160E074E184E090E0E1
:101B90000E94172660E086E090E00E94F9256FEF32
:101BA00087E090E00E94F92540E050E0BA0188E02B
:101BB00090E00E940B2660E08DE090E00E94F92505
:101BC00040E050E0BA0188E190E00E940B2660E01E
:101BD00087E190E00E94F92540E050E0BA018CE1F5
:101BE00090E00E940B2660E070E080E290E00E94AE
:101BF000172640E050E0BA0188E190E00E940B26F1
:101C000080E00E9402150E9437150E94AA0D0895D7
:101C10000E94B20D0895682F8EE090E00E94F92591
:101C200008950E94D71D6093300270933102809313
:101C300032029093330260932C0270932D028093B2
:101C40002E0290932F02089581E008950E94240EA1
:101C5000089508950E94290E08950E94290E08955E
:101C60000E942D0E08950E94290E08950E94330EA1
:101C700008950E94290E08958FEC90E10E94C71BE1
:101C80000E94390E0E94360E08950E942A0E0E946C
:101C9000290E08950E94EB100E94DC0308950E9413
:101CA000C21D0E9447150E94B8110E944A0E0E9450
:101CB000300E0895AAE0B0E0E0E6FEE00C94922534
:101CC0000E94CE1187E2E82E82E0F82E670100E044
:101CD000F60111916F01802F0E94061181270F5F7D
:101CE000053019F08823A1F322C0811120C00E9481
:101CF000CB1D8C01809125029091260208171907AF
:101D000009F450C08FEF89838A831B820E94CB1D08
:101D10008160782F9D838C8349815A816B818D816D
:101D20000E94080410932602009325023BC0809174
:101D3000340281FD0E940C110E94260EA82E10E094
:101D4000812F0E940611B82EF701C080C82611F11C
:101D500000E0DD24D3948C2D8D21B1F0AA20A1F0D8
:101D60000E831F8391E08B2D8D2109F490E09887DD
:101D70000E94CB1D8160782F9A8789874E815F8171
:101D800068858A850E9408040F5FDD0C043019F70E
:101D9000F701B0821F5FFFEFEF1AFF0A153081F6DF
:101DA0000E94110E0E94E9130E94EF032A96EAE0B6
:101DB0000C94AE25CF93DF930E94F00FEC018115B8
:101DC00020E59207E0F5811530E4930708F09FC005
:101DD000803E910528F58D3C910508F096C0883A23
:101DE000910570F4853A910508F085C08130910520
:101DF00009F47EC008F4DCC0049708F0DCC0D8C049
:101E0000813C910508F0D4C0C85AD0E0CC0FDD1F4A
:101E1000C85BDE4F0990D881C02DCE019464CCC040
:101E2000811540E2940708F0B8C0811551E095078C
:101E300008F0C1C0883E910508F4BDC0B9C0803625
:101E400062E5960720F5803472E5970708F06CC0CC
:101E5000C03282E5D80708F05EC0C11592E5D90707
:101E600008F489C02C2F2695269560E2269F9001C4
:101E70001124C37081E090E002C0880F991FCA95B9
:101E8000E2F7E901C82BD92BCE019D6895C0803AB5
:101E900022E59207E0F48F71C03832E5D30708F0ED
:101EA00059C08695869570E2879F900111249C2FDA
:101EB0009370C1E0D0E0AE0102C0440F551F9A9567
:101EC000E2F7EA01DA68C9018C2B9D2B75C0803CD2
:101ED00042E5940708F445C0803E924508F068C08A
:101EE000CF71DD27DC2FCC27CE01806F906A64C0D4
:101EF00081E090E061C0C55AD0E0C658DE4F8881CD
:101F0000C82FD0E0CE01906457C0906555C0DF70F7
:101F1000CE01906A51C0CF718C2F90E0D82FCC2782
:101F2000CE01816F906A48C08F718695869570E268
:101F3000879FA00111249C2F937021E030E0B9010C
:101F400002C0660F771F9A95E2F7CB019C68842B3D
:101F5000952B32C090E0D82FCC27CE01846F906AA9
:101F60002BC08F710E948C108F7190E0D82FCC27DE
:101F7000CE01906221C08C2F8F710E948C1095E051
:101F8000D695C7959A95E1F7CF70D0E0DC2FCC2796
:101F9000D069BE01682BCB010FC08D2F8F710E94BD
:101FA0008C10DD27D0628F719E01382BC90104C0CF
:101FB00080E090E001C0CE01DF91CF9108957530AF
:101FC00038F4643028F4462F672F0E94021A0895CF
:101FD00080E090E008950E94DF0F0E94DA0E0895DD
:101FE0008238910569F1B0F48133910509F475C027
:101FF00048F48932910509F467C08A32910509F4E1
:1020000071C008958533910509F459C0893391054C
:10201000B9F00895833E910589F138F4803E910529
:10202000D1F0823E910529F10895863E9105C9F1CE
:10203000873E9105D9F1843E910509F06CC027C017
:102040002091770220FD57C021FD55C020917802D4
:1020500023FD5BC008958091770280FD48C0809188
:10206000780280FF48C08091770284FD46C083EEED
:1020700051C08091770282FF3CC0F5CF80917702FA
:1020800082FD37C08091780280FD35C0ECCF809111
:10209000780281FF36C08091770284FD2EC087EEE2
:1020A00039C08091770283FF2AC0F5CF80917702F3
:1020B00083FD25C08091780281FD23C0ECCF809103
:1020C000770285FD22C01FC08091770285FD1BC06D
:1020D0008091780283FF19C00AC08091770286FD43
:1020E00016C017C08091770286FD13C010C089E327
:1020F00011C082EE0FC080EE0DC080E00BC086EEF6
:1021000009C084EE07C085E305C089E203C08AE206
:1021100001C081E390E008959091770292FF0DC095
:10212000282F2871283019F4877F846006C0282F53
:102130002471243011F48B7F886093FF0DC0282F09
:102140002871283119F4877E846106C0282F2471F4
:10215000243111F48B7E88612091780220FF0DC01C
:10216000382F3871383019F4877F816006C0382FD6
:102170003171313011F48E7F886021FF0DC0282F1E
:102180002871283119F4877E816106C0282F2171BA
:10219000213111F48E7E886194FD877E089580E060
:1021A00008950E946E0D08950E94CE118FE39CE960
:1021B0000197F1F700C000000E94CE1180E00E945C
:1021C000061180FF04C00E94D1100E94181E0895BD
:1021D0000E94D41008950E94750D811102C00E94C2
:1021E000080E0E94810D809334020E948B0D909303
:1021F0007802809377020E94E8100E94860D0E9468
:1022000055088091A7010E946A080895E82FF0E020
:10221000E258FD4F80810895089580EA8A95F1F78C
:10222000089500C008950E940D11089508950E9418
:10223000161108950E94171108950E94161108950D
:102240000E941D110895F894E82FE295EF70F0E0D8
:1022500031A1282F2F7081E090E001C0880F2A95CE
:10226000EAF7982F9095932391A392A1892B82A3AB
:10227000789408950F931F93CF93DF93C1E8D1E033
:1022800089918F3F11F00E94231181E0C638D80751
:10229000B9F7CDE7D1E001E811E089918F3F11F066
:1022A0000E9423110C171D07C1F7DF91CF911F91D9
:1022B0000F910895A0E0B0E0E0E6F1E10C949425E0
:1022C0008C01C62FD0E0CE018F579E4F7C01FC01C0
:1022D00090819F3F09F447C0D62EF894E92FE295EC
:1022E000EF70F0E081A19F7021E030E001C0220F8B
:1022F0009A95EAF7822B81A382A12095282322A315
:1023000078940E941111EDE7F1E041E851E031E0ED
:10231000C12C21912F3F89F0A22FA295AF70B0E080
:1023200090968C9190E02F7002C0959587952A9594
:10233000E2F780FD02C0832F01C080E0C82A330F7E
:102340004E175F0731F7F70180818F3F11F00E9430
:10235000231161E0C11001C060E08D2D0E941311B6
:10236000C00FD11FC882CDB7DEB7E8E00C94B0250E
:102370000E943A1185E0EEE7F2E0DF01982F1D920E
:102380009A95E9F7E9E7F2E0DF011D928A95E9F70E
:1023900085E00E9409120E943F030895A5E0B0E085
:1023A000E4EDF1E10C9497258E010F5F1F4F85E05E
:1023B000F80111928A95E9F7F12C6F2DC8010E945E
:1023C0005A11F394F5E0FF12F8CF45E050E0B80160
:1023D00089E792E00E94D52521E0009709F420E0EA
:1023E000892B41F085E0F801A9E7B2E001900D9258
:1023F0008A95E1F745E06EE772E089E792E00E9496
:102400000A12182F0E944203812F2596E5E00C94B2
:10241000B3250895EF92FF920F931F93CF93DF930D
:102420007C018B01C42F222349F081E08093370285
:102430000E94CB1D90933602809335028091370223
:10244000811102C080E01AC080913502909136025D
:102450000E94E31D0597B0F3D0E0AE01B701C801BB
:102460000E94D525892B39F0AE01B701C8010E9421
:10247000E22581E001C080E010923702CDB7DEB7DF
:10248000E6E00C94B2250E94CB1F0E944F0E0E94E2
:10249000D81F08950E94DD1F0E945A0E0E94F71F48
:1024A00008950E94621D0E94B11F0E943C0E0E946E
:1024B00043120E944A120E94450EFBCF80913E02B9
:1024C00080FF06C06091070170E0660F771F26C08D
:1024D00081FF04C06091070184E005C082FF07C04E
:1024E0006091070188E0689FB001112417C09091A6
:1024F0003D029923D1F060910601961788F720914B
:10250000070188E0289F90011124929FA001939FCA
:10251000500D112470E0CA010E94692560387105D0
:1025200040F46115710519F406C068E070E0862F6B
:1025300008958FE7089581E0089580913E0280FF1D
:1025400008C06091030170E0759567957595679572
:1025500021C081FF06C06091030170E07595679509
:1025600019C082FF04C06091030170E010C0909117
:102570003C02992399F0609102019617A0F780918F
:102580000301899FC001112470E00E946925603811
:10259000710540F46115710519F406C061E070E041
:1025A000862F08958FE7089581E008958D3C21F4EA
:1025B0000E945E12819504C08E3C29F40E945E1236
:1025C0008093420208958F3C21F40E945E1281950F
:1025D00004C0803D29F40E945E1280934102089558
:1025E000893D19F40E949D1205C08A3D31F40E9474
:1025F0009D1281958093430208958B3D21F40E94A2
:102600009D12819504C08C3D29F40E949D128093F7
:10261000440208959FE2980F983078F421E030E06A
:10262000A90102C0440F551F9A95E2F7CA01909183
:102630004002892B8093400208958D3D21F48091C2
:102640003E0281600BC08E3D21F480913E0282608B
:1026500005C08F3D29F480913E02846080933E0244
:1026600008958D3C39F49091420297FF35C0109245
:10267000420259C08E3C29F4909142021916BCF3D3
:102680002BC0909141028F3C29F497FF25C01092F6
:10269000410249C0803D19F41916CCF31DC0909138
:1026A0004302893D29F41916BCF4109243023BC041
:1026B0008A3D19F497FF10C0F8CF8B3D39F4909103
:1026C000440297FF09C0109244022DC08C3D21F4B2
:1026D000909144021916BCF39FE2980F983080F451
:1026E00021E030E0A90102C0440F551F9A95E2F79E
:1026F000CA0180959091400289238093400213C0C3
:102700008D3D21F480913E028E7F0BC08E3D21F4E1
:1027100080913E028D7F05C08F3D29F480913E025D
:102720008B7F80933E0280914102811106C080918F
:102730004202811102C010923D0280914302811138
:1027400006C080914402811102C010923C0208959B
:102750000E94CB1D20914102211104C02091420210
:10276000222321F090933B0280933A02209143026E
:10277000211104C020914402222321F090933902B8
:10278000809338028FE392E00E94F81B0895EFE3F4
:10279000F2E086E0DF011D928A95E9F710923D0292
:1027A00010923C0210923E020895FC018281811138
:1027B0000DC0838181110AC08481811107C091E01D
:1027C0008581811101C090E0892F01C081E0817075
:1027D0000895A6E0B0E0EFEEF3E10C94992586E0D1
:1027E000EFE3F2E0DE01119601900D928A95E1F798
:1027F000109241021092420210924302109244023F
:102800008B81811104C08C81882309F45FC0809181
:102810003A0290913B020E94E31DAC0190913D026F
:10282000992339F02091080130E02417350758F03A
:102830004DC0209109018AE0289F9001112424179E
:10284000350718F043C09F3F19F09F5F90933D02FA
:102850001B81112361F00E945E12111614F09FEF8C
:1028600001C091E0989F902D1124909341021C810A
:10287000112361F00E945E12111614F09FEF01C047
:1028800091E0989F902D1124909342023091410243
:102890003323E1F0209142022223C1F045EB3403BF
:1028A000C0011124992319F09093410203C081E0E3
:1028B0008093410235EB2303C0011124992319F0C1
:1028C0009093420203C081E0809342028D81811186
:1028D00004C08E81882309F45FC0809138029091F2
:1028E00039020E94E31DAC0190913C02992339F01A
:1028F0002091040130E02417350758F04DC0209195
:1029000005018AE0289F900111242417350718F04B
:1029100043C09F3F19F09F5F90933C021D8111239C
:1029200061F00E949D12111614F09FEF01C091E01A
:10293000989F902D1124909343021E81112361F0E2
:102940000E949D12111614F09FEF01C091E0989F14
:10295000902D112490934402309143023323E1F0EF
:10296000209144022223C1F045EB3403C00111241D
:10297000992319F09093430203C081E080934302AE
:1029800035EB2303C0011124992319F090934402DD
:1029900003C081E080934402BE016F5F7F4F8FE3ED
:1029A00092E00E94141D811105C08FE392E00E9405
:1029B000D51381110E94A81386E0FE013196AFE382
:1029C000B2E001900D928A95E1F72696E3E00C942F
:1029D000B52582E290E00E94EB25823281F483E209
:1029E00090E00E94EB25823151F484E290E00E9455
:1029F000EB2591E0883009F090E0892F01C080E05C
:102A000081700895CF93C82F811102C06FEF01C06C
:102A100062E282E290E00E94F925C11102C06FEFEC
:102A200001C062E183E290E00E94F925C11102C079
:102A30006FEF01C068E084E290E00E94F925CF9139
:102A40000895089585E290E00E94EB25682F70E0DC
:102A500080E090E008950895CF93C62F0E942B1533
:102A60006C2F85E290E00E94F925CF91089580E0D7
:102A70000E94021560E070E0CB010E942C150E94BC
:102A800097190E94571A81E00E94021508950E942A
:102A900021150E9422150E942B150E94E914811114
:102AA00002C00E94371508950895CF93FB01C2819B
:102AB000CC23E9F09C01225037472031310520F426
:102AC00082500E94671A0CC08115F7E79F0751F4E6
:102AD00081E00E947F0843E062E081E00E943503CC
:102AE000C0E018C081309747A9F482E0F2CF811589
:102AF000E7E79E0711F481E004C08130974749F46D
:102B000082E00E948B0843E062E081E00E9435038E
:102B100001C0C1E08C2FCF9108952FEFFC012083DD
:102B200008950E948D15089580E00895EF92FF9218
:102B30000F931F93CF93DF93EC01062F0E94941500
:102B40008111B1C0E8818E2F90E0FC013197E33113
:102B5000F10508F0A2C0EE59FF4F0C947D251982B3
:102B60008BE05EC08981823089F030F4813009F0D9
:102B700094C00E94D71D0CC0833079F0843009F0D6
:102B80008CC01A821B821C821D8289C00E94221561
:102B90009A838B837C836D8382C07E0182E0E80E02
:102BA000F11C10E0812F0E940611F70181937F0133
:102BB0001F5F1530B9F773C08981823039F08530D5
:102BC00009F06BC08A810E94541569C06A817B81BB
:102BD0008C819D810E9483250E942C1560C04B81B1
:102BE0006A8189810E945B199C838D8358C02C81E6
:102BF0003D813227232732274B816A8189810E94B8
:102C00007C194DC00E9497194AC0602FCE010E94C6
:102C1000911545C00E940E1A24C00E94101A998373
:102C20008A833DC06B8170E089819A81AE014C5FDF
:102C30005F4F9827892798270E94131A30C06B810D
:102C400070E089819A81AE014C5F5F4F9827892798
:102C500098270E94361A23C00E94571A20C00E944B
:102C6000481989831CC06B8170E089819A81AE010B
:102C70004C5F5F4F9827892798270E94C2190FC081
:102C80006B8170E089819A81AE014C5F5F4F98271C
:102C9000892798270E94E31902C08FEF8883602F4D
:102CA000CE010E94A01ECDB7DEB7E6E00C94B2259F
:102CB000CF93DF93FC01DB0112968C91882309F4FA
:102CC000DDC09F0130572332310508F0D8C0EF0135
:102CD0000E948B0D9093780280937702FE01E15061
:102CE000F047E232F10520F4EB58FF4F0C947D25BC
:102CF000809177028160AAC0809178028860B2C01A
:102D0000809177028260A2C08091770220C080917A
:102D1000770288609BC0809178021EC08091780203
:102D20008260A0C080917702806190C0809177021C
:102D300080628CC080917702806488C00E94F9070D
:102D400080917702806882C0809177028860846079
:102D50007DC0809178028260816084C0809177021A
:102D60008E7F74C080917802877F7CC080917702CB
:102D70008D7F6CC08091770220C080917702877F21
:102D800065C0809178021EC0809178028D7F6AC0F4
:102D9000809177028F7E5AC0809177028F7D56C0D6
:102DA000809177028F7B52C00E94F9078091770251
:102DB0008F774CC080917702877F8B7F47C080914F
:102DC00078028D7F8E7F4EC08091770282FB222712
:102DD00020F991E0922790FB82F990FB83F936C0AD
:102DE00080917802982F909591708E7F892B90FB1F
:102DF00081F938C08091770286FB222720F991E083
:102E0000922790FB86F922C00E94F90780917702F1
:102E100087FB222720F991E0922790FB87F916C0C3
:102E200081E001C080E00E940B0E1EC080917702FD
:102E300084FB222720F991E0922790FB84F906C0B9
:102E400080917702982F909590FB80F9809377027C
:102E50000BC08091780283FB222720F991E0922712
:102E600090FB83F9809378028091770290917802A9
:102E70000E94900D0E94F90780E001C081E0DF917F
:102E8000CF910895A0E0B0E0E8E4F7E10C94952537
:102E9000E82FF0E0E259FD4FD490282F2695269593
:102EA000269530E0F901E25FFC4F0491877010E055
:102EB000082E02C0159507950A94E2F701701127B4
:102EC000F901E250FD4FE490F12C082E02C0F59478
:102ED000E7940A94E2F791E0E922FF24F901E25134
:102EE000FD4FC491D0E002C0D595C7958A95E2F711
:102EF000C170DD270115110519F081EE0E945904FA
:102F0000E114F10419F086EE0E9459048D2D0E94FF
:102F10008C05E114F10419F086EE0E9408050115F4
:102F2000110519F081EE0E940805CD2B19F08CE2F5
:102F30000E948C05CDB7DEB7E7E00C94B125EF9287
:102F4000FF920F931F93CF93DF93EC01162F0AE0AC
:102F50008881882309F455C0813009F043C08981F4
:102F6000813041F47E0182E0E80EF11C8A810E94EA
:102F70008C0509C0823049F47E01E2E0EE0EF11CBE
:102F80008A810E945904E7012FC0833041F47E01F9
:102F9000F2E0EF0EF11C8A810E940805F4CF843024
:102FA00011F0219621C02A81229680E090E030E045
:102FB000205331092A30310558F4089FA001099F98
:102FC000500D1124C901840F951F21962881EFCF40
:102FD000009751F0EFE9FFE03197F1F700C00000F2
:102FE0000197F6CF0E9442172196812F882309F47A
:102FF000AFCFEFE9FFE03197F1F700C0000081505B
:10300000F5CFCDB7DEB7E6E00C94B225893289F171
:10301000F0F4843171F1B0F4873009F077C081E0C9
:103020008093090184E1809308018AE0809307017D
:103030008EE18093060188E08093030188E280930B
:10304000020164C092EE980F9A30F0F05FC08035B4
:1030500009F444C028F48F3409F058C08AE03FC016
:10306000813529F0823509F051C081E038C08FEFF9
:1030700036C080914702882379F11092470210925E
:1030800046021092450242C08D5180934702833020
:1030900099F038F4813069F08230D9F488E091E019
:1030A0000DC0853099F078F0863099F482E091E097
:1030B00005C089E091E002C087E091E0909346026C
:1030C0008093450223C086E091E0F8CF83E091E051
:1030D000F5CF109247021AC080E0089586EFE09184
:1030E0004502F0914602309789F02081082E000CAD
:1030F000990B820F911D8F3F910519F014F08FEFFE
:1031000004C097FF02C0108201C0808381E008954F
:10311000482F50E0FA013597EF33F10508F068C009
:10312000E956FF4F0C947D250E94080E5DC08091EA
:103130003402817F8E7F8093340281E08093480245
:1031400008950E94540350C080913402982F9095A6
:10315000917090FB80F980933402911145C0897F72
:10316000877F10C08091340281FB222720F991E0F3
:10317000922790FB81F9809334029923A9F18091E1
:1031800034028160809334022FC08091340282FB2C
:10319000222720F991E0922790FB82F9ECCF8091D1
:1031A000340283FB222720F991E0922790FB83F9D8
:1031B000E2CF0E94F9078091770287FB222720F94E
:1031C00091E0922790FB87F9809377020DC0895395
:1031D00001C08D5191E001C0990F8A95EAF7892FBE
:1031E0000E9455080E94F90781E0089581E0F8CF18
:1031F00080E0089580E008950E94FA180895CF9322
:10320000C82F80914802813069F038F08230C1F5D2
:103210008C2F0E94061881E039C00E94840C8232F3
:1032200089F504C00E94840C823261F48C2F0E94C4
:10323000FC18811104C08C2F0E9488181FC081E0E7
:1032400090E01CC08C2F0E94FA18811116C0C43166
:1032500089F058F4CB3089F0C031B1F482E080932A
:10326000480288E30E94061808C0C93219F0C83322
:1032700021F00AC01092480207C081E0817006C0A8
:103280001092480280E002C080E0F8CFCF9108950C
:1032900084E0089550E0440F551F28E0629F400DE0
:1032A000511D11249A0168E2869F200D311D1124C1
:1032B000C901869608950F931F93CF93DF938430AF
:1032C000A0F4653090F4443080F40E944A198C01D7
:1032D0000E94EB2590E0D82FCC27C80101960E94D0
:1032E000EB259E01282BC90102C080E090E0DF9110
:1032F000CF911F910F9108950F931F93CF93DF9359
:10330000843080F4653070F4443060F4E9010E9448
:103310004A198C016D2F0E94F9256C2FC801019666
:103320000E94F925DF91CF911F910F9108950F937E
:103330001F93CF93DF93C0E0D0E010E000E00E9445
:10334000A90290E0C817D9073CF4402F612F8C2FB9
:103350000E94AB029C0102C021E030E0402F612FAF
:103360008C2F0E947C190F5F043049F71F5F1530C6
:1033700029F72196C430D10501F7DF91CF911F9134
:103380000F910895EF92FF920F931F93CF93DF93C6
:10339000EA017A01E60EF71E8C01C8018696CE1569
:1033A000DF0561F0003A110520F40E94EB258883C7
:1033B00001C0188221960F5F1F4FEFCFCDB7DEB748
:1033C000E6E00C94B225EF92FF920F931F93CF93F8
:1033D000DF93EA017A01E60EF71E8C01C80186969A
:1033E000CE15DF0551F0003A110518F468810E94EE
:1033F000F92521960F5F1F4FF1CFCDB7DEB7E6E07D
:103400000C94B225843038F4653028F4443018F434
:103410000E945B19089580E090E0089580E108958E
:103420008AE393E00895EF92FF920F931F93CF9357
:10343000DF93EA017A01E60EF71E8C01C8018A5378
:103440009F4FCE15DF0569F00A3323E0120720F401
:103450000E94EB25888301C0188221960F5F1F4FC1
:10346000EDCFCDB7DEB7E6E00C94B225EF92FF9238
:103470000F931F93CF93DF93EA017A01E60EF71EB5
:103480008C01C8018A539F4FCE15DF0559F00A33CE
:1034900023E0120718F468810E94F92521960F5F36
:1034A0001F4FEFCFCDB7DEB7E6E00C94B225CF9338
:1034B000DF93C6ECD0E060E0CE010E94F9252196B2
:1034C000C11584E0D807B9F7DF91CF910895A8E03E
:1034D000B0E0EDE6FAE10C949025F82E8FE08F1520
:1034E00008F474C08FEF93E00E94EB2581116EC049
:1034F00006EC10E0FF2071F0011594E0190709F4C3
:1035000065C0C8010E94EB25811101C0FA940F5FCC
:103510001F4FF0CFFE0131966F0188E011928A951E
:10352000E9F77801FFEFEF1AFF0AC8010E94EB25C7
:1035300089831A82882309F449C0813009F040C088
:10354000580182E0A80EB11CC7010E94EB258A83B6
:103550008823E1F19FEF980F933060F4780193E0B6
:10356000E90EF11CC5010E94EB258B83882371F1C4
:103570001C8226C0843019F54E01E3E08E0E911CAA
:1035800002E010E07501FFEFEF1AFF0AC5010E948B
:10359000EB25F40181934F018823C1F08C3741F46E
:1035A000E2E0F0E0EC0FFD1FE00FF11F108208C019
:1035B0000F5F1F4F57010730110521F707C0750135
:1035C00060E0C6010E949F178701ABCF2896ECE010
:1035D0000C94AC25CF93DF9386319C4741F5EB01EA
:1035E0000E94840C982F8A81209100013091010162
:1035F000882379F09A7A81E009F480E08093490287
:10360000911102C069E201C065E3C9010E94E61C94
:103610000AC080914902811102C069E201C065E3DC
:10362000C9010E94F41C0E94C80C80E001C081E026
:10363000DF91CF9108950F931F93CF93DF93C42F02
:10364000D22FFC0182818823B1F040934C020E946A
:10365000CB1D90934B0280934A0280E28C0F8830FE
:1036600008F04DC0C77081E001C0880FCA95EAF725
:103670000E94960544C080914C02481330C080914E
:103680004A0290914B020E94E31D883C910538F557
:1036900010E21D0FCD17B9F080E28C0F883040F496
:1036A000C77081E001C0880FCA95EAF70E949D05A6
:1036B000183010F581E09D2F977001C0880F9A9502
:1036C000EAF70E949605802F0E948C051830B8F406
:1036D000D77081E001C0880FDA95EAF70AC080E26E
:1036E0008C0F883060F4C77081E001C0880FCA95E4
:1036F000EAF70E949D0503C0802F0E948C05DF9190
:10370000CF911F910F9108950F93FC01E851FC4751
:10371000E730F10590F5CB01EA52FF4F0C947D257F
:1037200006E221EE41EE6AE17CE723C007E225EEE6
:1037300045EE6BE17CE71DC006E221EE40EE68E15C
:103740007CE717C007E225EE44EE69E17CE711C093
:1037500006E221EE42EE6CE17CE70BC007E225EECB
:1037600046EE6DE17CE705C008E221E045EE6EE142
:103770007CE70E941B1B80E008C0FB01828188233C
:1037800019F010924C0201C081E00F9108959093BE
:10379000970180939601089590935202809351026D
:1037A0000895E0915102F0915202309729F0019072
:1037B000F081E02D0995089580E00895FC01A09125
:1037C0005102B0915202109791F08091120188231A
:1037D00041F08091770287FF04C08081818386E079
:1037E0008083CF011296ED91FC911397099508956E
:1037F000E0915102F0915202309739F022E0DC0161
:103800002C930480F581E02D09950895A3E0B0E0A4
:10381000ECE0FCE10C949A2520914F02309150028B
:1038200028173907A1F09093500280934F02E0913E
:103830005102F0915202309751F023E029839B838B
:103840008A830680F781E02DCE01019609952396A3
:10385000E2E00C94B625A3E0B0E0E1E3FCE10C94D7
:103860009A2520914D0230914E0228173907A1F078
:1038700090934E0280934D02E0915102F0915202DA
:10388000309751F024E029839B838A830680F78157
:10389000E02DCE01019609952396E2E00C94B62521
:1038A000FC01329680911201882331F080917702D9
:1038B00087FF02C09EE101C096E080E0915028F0B1
:1038C00021912223D9F38F5FF9CF0895662351F117
:1038D000209112012223E9F02091770227FF19C0DD
:1038E000462F4695469546954E31E0F4677021E0A7
:1038F00030E002C0220F331F6A95E2F7FC01E40FAB
:10390000F11D828190E02823392381E0232B69F483
:1039100009C0FC01329608962191621729F0E81738
:10392000F907D1F780E0089581E008959C01FC013A
:1039300032969FEF80E04191461789F09F3F19F43E
:10394000411101C0982F8F5F8630A9F79F3F39F052
:10395000F901E90FF11D97FDFA9562830895089525
:103960009C012A5F3F4FFC014281461301C0128235
:10397000019682179307B9F70895262F2695269565
:1039800026952E3168F4FC01E20FF11D677021E0ED
:1039900030E001C0220F6A95EAF78281282B22834A
:1039A0000895262F2695269526952E3170F4FC0134
:1039B000E20FF11D677021E030E001C0220F6A952F
:1039C000EAF720958281282322830895209112010D
:1039D000222339F02091770227FF03C00E94BD1CEB
:1039E00008950E94961C089520911201222339F017
:1039F0002091770227FF03C00E94D11C08950E94E6
:103A0000B01C089520911201FC013296222331F05E
:103A10008091770287FF02C08EE101C086E0DF015E
:103A20001D928A95E9F7089546E050E00E94D52559
:103A300021E0892B09F420E0822F089508950E9447
:103A40001E1D089583E0809353020E941F1D089558
:103A5000811102C081E001C082E0809353020E9484
:103A60001F1D08950E94281D089581E08093530230
:103A70000E941F1D08950E94351D089508950E94FB
:103A80003E1D08950E943F1D08950E943E1D089509
:103A90000E943E1D08950E943E1D0895CF930E94EE
:103AA000481D0E94CE110E94451DC0E08C2F0E942F
:103AB0000611811104C0CF5FC530C1F701C081E09C
:103AC000CF91089585B7806885BF85B7806885BF29
:103AD00008951F920F920FB60F9211248F939F9308
:103AE000AF93BF9380915402811113C080918302E0
:103AF00090918402A0918502B09186024196A11D09
:103B0000B11D8093830290938402A0938502B093A9
:103B10008602BF91AF919F918F910F900FBE0F9032
:103B20001F90189580918B02843031F10E94BC0364
:103B30001092540220E488E190E00FB6F894A89522
:103B4000809360000FBE2093600083B7817F846004
:103B500083BF83B7816083BF7894889583B78E7F56
:103B600083BF0FB6F894A895809160008861809318
:103B70006000109260000FBE08950E94F9070E9435
:103B8000C103089582E084BD93E095BD9AEF97BD8F
:103B900080936E0008952FB7F894809183029091DE
:103BA0008402A0918502B09186022FBF08952FB79D
:103BB000F8946091830270918402809185029091C3
:103BC00086022FBF08959C014FB7F894809183021D
:103BD00090918402A0918502B09186024FBF821B12
:103BE000930B089578941F920F920FB60F921124A1
:103BF0008F939F93AF93BF938091830290918402A0
:103C0000A0918502B09186020196A11DB11D8093FD
:103C1000830290938402A0938502B0938602BF91A1
:103C2000AF919F918F910F900FBE0F901F9018959D
:103C300081E08093E00080E28093D8001092C90078
:103C40008FE19EE40197F1F700C0000087E090EB60
:103C5000DC018093940290939502A0939602B09316
:103C600097029CE088E10FB6F894A89580936000D5
:103C70000FBE90936000FFCF9CE088E10FB6F894F0
:103C8000A895809360000FBE90936000FFCF809155
:103C9000750208959B0190918B029430F1F48F701E
:103CA0008093E9008FEF9091E800815095FD06C068
:103CB00095ED9A95F1F700008111F5CF8091E8001C
:103CC00085FF0BC0BA01C90140E050E00E94962078
:103CD0008091E8008E778093E800089543E050E0FB
:103CE000BC0184E00E944A1E089546E050E0BC01F9
:103CF00084E00E944A1E0895CF93DF93EC018091E7
:103D00001201811105C048E050E0BE0181E00BC006
:103D10008091770287FF03C040E284E002C048E060
:103D200081E050E0BE010E944A1E80E2FE01A5E54E
:103D3000B2E001900D928A95E1F7DF91CF9108955D
:103D4000603231F4BC0140E250E082E00E944A1E41
:103D5000089580918A02811109C00E9466220E9402
:103D6000C3228091E20084608093E2000895109263
:103D70008A0208950E943B1D08956091870281E0A8
:103D8000611101C080E00E94221D089590918B0274
:103D900081E0943009F080E0609187020E94281D44
:103DA000089542E061EC81E00E94DF2142E261EC93
:103DB00084E00E94DF2142E261EC82E00E94DF2188
:103DC00042E260EC83E00E94DF2190918B0281E06F
:103DD000943009F080E0609187020E94321D0895BE
:103DE00080918D02833009F463C030F4813071F02A
:103DF000823009F49DC008958A3009F489C08B305F
:103E000009F46EC0893009F0ABC020C080918C02EB
:103E1000813A09F0A5C08091E800877F8093E8008F
:103E20008091900290919102892B21F460E285E5C6
:103E300092E003C060E080E090E070E00E9420210A
:103E40008091E8008B778093E800089580918C0240
:103E5000813209F085C08091900290919102009783
:103E600019F0029709F07CC08091E800877F809369
:103E7000E8008091E80082FD05C080918B028111ED
